:020000040800F2
:100000000004022001020008C90E0008CD0E0008FD
:10001000210F0008CD0E0008F50E000803020008AD
:10002000030200080302000803020008C9300008A8
:10003000030200080302000803020008030200088C
:10004000030200080302000803020008030200087C
:100050000302000803020008213300084D330008A2
:1000600079330008A5330008D133000803020008E3
:10007000030200080302000803020008030200084C
:10008000030200080302000803020008030200083C
:10009000030200080302000803020008FD33000801
:1000A000030200080302000803020008030200081C
:1000B000453100080302000803020008030200089B
:1000C00003020008030200080302000803020008FC
:1000D00003020008030200080302000803020008EC
:1000E0006534000803020008030200080302000848
:1000F00003020008030200080302000803020008CC
:1001000003020008030200080302000803020008BB
:1001100003020008030200080302000803020008AB
:10012000030200080302000803020008030200089B
:10013000030200080302000803020008030200088B
:10014000030200080302000803020008D527000884
:10015000030200080302000803020008030200086B
:10016000030200080302000803020008030200085B
:10017000030200080302000803020008030200084B
:10018000030200080302000803020008030200083B
:10019000030200080302000803020008030200082B
:1001A000030200080302000803020008030200081B
:1001B000030200080302000803020008030200080B
:1001C00003020008030200080302000803020008FB
:1001D00003020008030200080302000803020008EB
:1001E00003020008030200080302000803020008DB
:1001F00003020008030200080302000803020008CB
:1002000002E000F000F8FEE772B6394880F3088893
:10021000384880F3098838484EF60851CEF200017C
:10022000086040F20000CCF200004EF63471CEF2CD
:1002300000010860BFF34F8FBFF36F8F40F20000E3
:10024000C0F2F0004EF68851CEF200010860BFF314
:100250004F8FBFF36F8F4FF00000E1EE100A4EF6A4
:100260003C71CEF200010860062080F31488BFF3D1
:100270006F8F01F037FF02F0AFFE4FF055301F498E
:100280001B4A91423CBF41F8040BFAE71C49194A4A
:1002900091423CBF41F8040BFAE71A491A4A1B4B3A
:1002A0009A423EBF51F8040B42F8040BF8E70020D5
:1002B0001749184A91423CBF41F8040BFAE701F094
:1002C00055FF02F0F3FE144C144DAC4203DA54F81F
:1002D000041B8847F9E700F03FF8114C114DAC4280
:1002E00003DA54F8041B8847F9E701F03DBF00002A
:1002F0000004022000240220000000080000022068
:100300000004022088380008002402205024022023
:100310005024022058300220000200080002000889
:1003200000020008000200082DE9F04F2DED108AB0
:10033000C1F80CD0D0F80CD0BDEC108ABDE8F08F1D
:10034000002383F311882846A047002001F052FBC8
:1003500001F002FB00DFFEE770B56FF00F03204CE9
:1003600000256FF07F0623700323A57063701E23A2
:10037000E57025716571A571E57125726672A372CC
:10038000E57200F007FD20B10E2325726672A3729C
:10039000E57201F069FE044601F09EFE0546D0B903
:1003A000104B9C4219D001339C4241F2883412BF59
:1003B000054600240125002001F060FE0DB100F08B
:1003C000B7F800F055FD00F039FC204600F050F978
:1003D00000F0AEF8F9E70024EDE70446EBE700BFD4
:1003E00050240220010007B008B500F0C9FBA0F1BD
:1003F00020035842584108BD054B07B51B88022110
:1004000001A8ADF8043000F009FC03B05DF804FB6E
:1004100048350008064991F8243033B100230822FA
:10042000086A81F8243000F02DBC0120704700BF1D
:10043000702402202DE9F84F234C054688461746C4
:1004400094F824308BBB2E46DFF87C90002F38D0F8
:1004500094F824A0BAF1000F05D12022FF214846CC
:10046000266200F0F3FCCAF10805414604EB8A005D
:10047000BD4228BF3D465FFA85FBAD00A7EB0B07E9
:100480002A462E4400F0BAFC94F82430A844FFB267
:100490009B445FFA8BFBBBF1080F84F824B0D5D1E5
:1004A000FFF7B8FF0028D1D108E0266A06EB8306E3
:1004B000B042C9D0FFF7AEFF0028C4D10020BDE88C
:1004C000F88F0120BDE8F88F7024022010B520239A
:1004D00083F311881248C3680BB101F011FB0023AC
:1004E000104A4FF47A710E4801F0CEFA002383F3DC
:1004F00011880D4C236813B12368013B23606368A6
:1005000013B16368013B6360084B1B7833B96368C0
:1005100023B9022000F068FC3223636010BD00BFE5
:100520005C240220CD040008A0250220982402208B
:10053000454B46492DE9F04153F8042F013201D1D2
:10054000BDE8F0818B42F7D1414C424B22689A4280
:1005500078D9414B9B6803F1006303F5C0339A429D
:1005600070D2002000F086FB02203C4B187000F097
:1005700033FC3B4B1A6C00221A64196E1A66196E12
:10058000596C5A64596E5A66596E596941F0800126
:100590005961596921F0800159615969196941F01E
:1005A00000511961196921F0005119611B6972B676
:1005B0002C4B2D490B601D682468BFF34F8FBFF390
:1005C0006F8F2A4BC3F88420BFF34F8F5A6922F4F0
:1005D00080325A61BFF34F8FD3F8802043F6E07E1C
:1005E000C2F3C906C2F34E32B707520102EA0E083F
:1005F00038463146013948EA000C00F14040B1F17B
:10060000FF3FC3F874C2F5D1203A12F1200FEDD1AB
:10061000BFF34F8FBFF36F8FBFF34F8FBFF36F8F5A
:100620005A6922F400325A610022C3F85022BFF303
:100630004F8FBFF36F8F202383F31188AD4685F36F
:1006400008882047BDE8F081FC7F01081C80010874
:1006500004800108FF7F0108502402209824022012
:10066000003802400080010808ED00E000ED00E0E5
:100670002DE9F04F99B0B34C2022FF21019010A832
:10068000A66800F0E3FBB04AA3461378A3B90121A2
:10069000AE481170C360202383F31188C3680BB187
:1006A00001F02EFA0023AA4A4FF47A71A74801F00C
:1006B000EBF9002383F31188019B13B1A54B019A39
:1006C0001A600023A44AA349019F99461C461D466F
:1006D000984613704B600292012000F07DFB002FC2
:1006E00000F012829B4B1B68002B40F00D8219B06A
:1006F000BDE8F08F0220FFF777FE002840F0FB8175
:10070000019BB9F1000F08BF1F46944B1B880221C3
:100710000BA8ADF82C3000F081FADDE74FF47A70C9
:1007200000F02EFA031E0393EADB0220FFF75CFEC3
:1007300082460028E4D0039B581E042800F2DD8185
:10074000DFE800F0030E1114170018A80523042198
:1007500040F8343D00F062FA54464FF0000856E08D
:1007600004217848F6E704217D48F3E704217D4819
:10077000F0E71C242046043400F07EFA04210B909C
:100780000BA800F04BFA2C2CF4D1E5E7002DB7D0E4
:10079000002CB5D00220FFF727FE0546002800F008
:1007A000AF8101206C4C00F065FA4FF00009022087
:1007B000207000F011FB5FFA89FA504600F06AFAE7
:1007C000074658B1504609F1010900F073FA0028B4
:1007D000F1D12C46A9460027634B97E701233E46FB
:1007E0000220237000F0EEFADBF808309E4206D2B9
:1007F000304600F041FA0130EBD10436F4E7002630
:10080000029BA9462C461E703746524B5E6000F094
:1008100025FB15B1002C18BF0027FFF7EDFD5BE7A6
:10082000002D3FF46DAF002C3FF46AAF0220029B15
:10083000187000F0D1FA322000F0A2F9B0F1000AED
:10084000C0F25E811AF0030540F05A8106EB0A03FC
:10085000DBF80820934200F25381BAF5807F00F262
:100860004F8155450DDA4FF47A7000F089F9049004
:10087000049B002BC0F24481049B3C4AAB540135DD
:10088000EFE7C820FFF7B0FD0546002800F03881EB
:100890001F2E11D8C6F1200410AB26F003003349F7
:1008A0005445184428BF5446224600F0A7FA224671
:1008B000FF212E4800F0CAFA4FEAAA0A2B49304617
:1008C0005FFA8AF2FFF7B6FD0446002800F01A81AD
:1008D00006EB8A0605469AE70220FFF785FD002809
:1008E0003FF40EAFFFF796FD00283FF409AF4FF03D
:1008F000000A5346DBF8082092451CD2BAF11F0FBC
:1009000012D8109A01320FD02AF0030218A90A4413
:1009100052F8202C0B92184604220BA90AF1040A63
:1009200000F012FB0346E5E75046039300F0A4F9FC
:10093000039B0B90EFE718A8042140F84C3D00F012
:100940006DF964E7502402209C2502205C240220DB
:10095000CD040008A0250220982402204A35000872
:1009600054240220582402204C3500089C240220E4
:1009700018A80023642140F8343D00F02BF900282A
:100980007FF4BEAE0220FFF72FFD00283FF4B8AE83
:100990000B9800F0A1F918AB43F8480D0421184654
:1009A000CDE718A80023642140F8343D00F012F987
:1009B00000287FF4A5AE0220FFF716FD00283FF4C3
:1009C0009FAE0B9800F096F918AB43F8440DE5E79D
:1009D0000220FFF709FD00283FF492AE00F090F9E5
:1009E00018AB43F8400DD9E70220FFF7FDFC0028C3
:1009F0003FF486AE0BA9142000F088F9824618A8AF
:100A0000042140F83CAD00F009F951460BA896E7E7
:100A1000322000F0B5F8B0F1000AFFF671AE1AF01E
:100A2000030F7FF46DAE0AEB0803DBF80820934256
:100A30003FF666AE0220FFF7D7FC00283FF460AE19
:100A40002AF0030AC244D0453FF4E1AE404608F123
:100A5000040800F011F904210A900AA800F0DEF859
:100A6000F1E74FF47A70FFF7BFFC00283FF448AE7F
:100A7000FFF7D0FC00283FF4AFAE109B01330CD041
:100A8000082210A90020FFF7D5FC00283FF4A4AEEF
:100A90002022FF2110A800F0D9F9FFF7ADFC37485C
:100AA00000F0AEFF23E6002D3FF42AAE002C3FF409
:100AB00027AE18A80023642140F8343D00F08AF8DE
:100AC000824600287FF41CAE0220FFF78DFC002830
:100AD0003FF416AE0390FFF78FFC41F28830574683
:100AE00000F08EFF0B9800F0EDF900F0B7F9039BD2
:100AF0001C461D46F0E5054689E64FF00008FFE577
:100B00002546FDE52C4667E6002000F039F8049004
:100B1000049B002BFFF6E3AD012000F053F9049B8A
:100B2000213B122B3FF6D8AD01A252F823F000BFB3
:100B3000F50600081D0700088D070008D906000803
:100B4000D9060008D906000821080008110A000883
:100B5000D908000871090008A3090008D109000894
:100B6000D9060008E9090008D9060008630A000848
:100B70000F080008D9060008A70A0008A08601008F
:100B8000114B37B51A780024014601328DF8074021
:100B9000D2B2012A11D80D48012203681D6A4FF410
:100BA0007A734B430DF10701A847012805D1084B83
:100BB0009DF807001C7003B030BD4FF4FA7000F0D0
:100BC0001FFF4FF0FF30F6E70024022070260220BE
:100BD000AC25022038B50E4B05461A780132D2B248
:100BE000012A0ED80B48042203681C6A4FF47A735A
:100BF0004B432946A047042803D10020064B187018
:100C000038BD4FF4FA7000F0FBFE4FF0FF3038BDF6
:100C10000024022070260220AC25022030B4054CAE
:100C20000A46014623682046DD69034BAC4630BCCA
:100C3000604700BF70260220A0860100F8B50A4C6C
:100C400000250A4E01F016F9094F2070306823780C
:100C5000834207D901F008F9336805440133BD42E6
:100C60003360F3D9F8BD00BFAD250220A8250220CE
:100C7000FF7F010001F0AAB900F1006000F5C0306B
:100C80000068704700F10060920000F5C03001F08C
:100C900037B90000054B1A68054B1B789B1A834235
:100CA00002D9104401F0E0B800207047A8250220C6
:100CB000AD25022038B5074D04462868204401F0D0
:100CC000DBF828B928682044BDE8384001F0ECB8CA
:100CD00038BD00BFA825022010F0030308D1B0F5ED
:100CE000806F05D800F10050A0F5712000687047B2
:100CF00000207047014BC058704700BF20F4F01F20
:100D0000014B1868704700BF002004E01F4BF0B58E
:100D10001E681F4BC6F30B02360C1F885D68BA4273
:100D200093F9084022D09F89BA4221D01F8BBA4242
:100D300006D102220C2404FB02335D6893F90840BB
:100D4000B6F5805F16D041F201039E4208BF5A24D7
:100D5000421E013D0B460A44934215D215F9016F1C
:100D6000581C4EB1034600F8016CF5E70022E1E79C
:100D70000122DFE74124EBE72C2582421D7001D9D7
:100D8000981C5C70401AF0BD1846FBE7002004E098
:100D900004240220094B5B88B3F5805F09D041F23F
:100DA0000102934207D10122054B03EB8203D8785D
:100DB00070470022F8E70020704700BF002004E0E1
:100DC00050350008022803D14FF48032014B9A615C
:100DD000704700BF00100240022802D10122014BDF
:100DE0009A61704700100240022804D1024A5369F8
:100DF00083F001035361704700100240002310B5D7
:100E0000934203D0CC5CC4540133F9E710BD000019
:100E100030B5441E14F9010F0B4658B193F9005038
:100E20000131854206D11AB993F90020801A30BDEC
:100E3000013AEFE7002AF7D1104630BD02460346DB
:100E4000981A13F9011B0029FAD17047024403468E
:100E5000934202D003F8011BFAE77047024B1A785D
:100E6000024B1A70704700BFAC25022000240220FC
:100E700038B5104D104C284600F002F9214628469E
:100E800000F02AF924680D48E26ED2F8043843F0E5
:100E90000203C2F8043800F0B3FD0949204600F00F
:100EA00029FAE26ED2F8043823F00203C2F80438BB
:100EB00038BD00BF702602200036000840420F00F7
:100EC0002836000870470000FEE7000000B59BB020
:100ED000EFF3098168226846FFF790FFEFF305837F
:100EE000034B9A6B9A6A9A6A9A6A9A6A9B6AFEE7B5
:100EF00000ED00E000B59BB0EFF309816822684681
:100F0000FFF77CFFEFF30583044B9A6B9A6A9A6AAA
:100F10009A6A9A6A9A6A9B6AFEE700BF00ED00E04F
:100F200000B59BB0EFF3098168226846FFF766FFC2
:100F3000EFF30583034B5A6B9A6A9A6A9A6A9A6A24
:100F40009B6AFEE700ED00E030B50A44074D914290
:100F50000BD011F8013B09245840013CF7D040F375
:100F600000032B4083EA5000F7E730BD2083B8ED43
:100F7000002304491A465A50C81808334260802B8F
:100F8000F9D17047B025022002684368114301601F
:100F900003B118477047000013B5446BD4F894347C
:100FA0001A681178042915D1217C022912D11979E6
:100FB000012312898B4013420CD101A904F14C008A
:100FC00001F080FED4F894440246019B2179206808
:100FD00000F0E0F902B010BD143001F003BE0000D3
:100FE0004FF0FF33143001F0FDBD00004C3001F034
:100FF000D5BE00004FF0FF334C3001F0CFBE0000F3
:10100000143001F0D1BD00004FF0FF31143001F079
:10101000CBBD00004C3001F0A1BE00004FF0FF320C
:101020004C3001F09BBE0000D0F8942438B5136812
:1010300005461978042901D0012038BD017C022918
:10104000FAD1127901205C8990400440F4D105F175
:10105000140001F063FD02460028EDD0D5F8945449
:101060004FF480732868697900F082F9204638BD12
:10107000406BFFF7D9BF00000020704770470000A9
:101080007FB5124B01250226044603600023057438
:1010900000F18402436029468360C3600C4B0290D8
:1010A000143001934FF48073009601F013FD094B47
:1010B00004F523722946019304F14C004FF4807328
:1010C0000294009601F0DAFD04B070BD843500088A
:1010D00071100008990F00080B68202282F3118814
:1010E0000A7903EB820210624A790D3243F822003A
:1010F0008A7912B103EB820318620223C0F89414B8
:101100000374002383F311887047000038B5037F10
:10111000044613B190F85430ABB90125201D0221CB
:10112000FFF732FF04F1140025776FF0010100F0A2
:101130008FFC84F8545004F14C006FF00101BDE8BD
:10114000384000F085BC38BD10B50121044604309C
:10115000FFF71AFF0023237784F8543010BD0000F6
:1011600038B504460025143001F0CCFC04F14C00E5
:10117000257701F09BFD201D84F854500121FFF7D5
:1011800003FF2046BDE83840FFF74EBF90F85C30C3
:1011900003F06003202B19D190F85D20212A0AD09A
:1011A000222A4FF000030ED0202A0FD1084A0265F0
:1011B0000722426504E0064B0365072343650023CD
:1011C00083650120704703654365F9E70020704798
:1011D00028240220D0F8943437B51A6804461178D0
:1011E00004291AD1017C022917D119790123128906
:1011F0008B40134211D100F14C05284601F016FE38
:1012000058B101A9284601F05DFDD4F89444024686
:10121000019B2179206800F0BDF803B030BD0000CB
:1012200000EB8103F7B51C6A05460E46F4B1202396
:1012300083F3118805EB8607201D08214C34FFF746
:10124000A3FEFB685B691B6813B1204601F048FDF3
:1012500001A9204601F036FD024648B1019B314606
:10126000284600F097F8002383F3118803B0F0BDFF
:10127000FB685A691268002AF5D01B8A013B1340AB
:10128000F1D105F15C02EAE70D3138B550F82140A3
:10129000DCB1202383F31188D4F8942413685279A5
:1012A00003EB8203DB689B695D6845B1042160182C
:1012B000FFF76AFE294604F1140001F039FC2046CC
:1012C000FFF7B2FE002383F3118838BD704700009A
:1012D00000F0D2BF012300F1240200F138010370B5
:1012E0000023436042F8043B8A421361FAD1038130
:1012F0004381704738B50446202383F311880025C5
:101300004160C560056145618561C561056200F0A8
:10131000C3FF0223237085F3118838BD70B500EB3D
:101320008103054650690E461446DA6018B1102252
:101330000021FFF78BFDA06918B110220021FFF7F3
:1013400085FD31462846BDE8704001F06FB80000C9
:10135000028902F001020281428902F00102428107
:101360000022026142618261C261026201F0F2B850
:10137000F0B4012500EB810447898D40E4683D43CA
:10138000A469458123600023A2606360F0BC01F082
:101390000DB90000F0B4012500EB810407898D40F0
:1013A000E4683D436469058123600023A2606360B3
:1013B000F0BC01F087B9000070B502230025044697
:1013C0000370A0F8645080F8665080F8675005817B
:1013D0004581C560056145618561C561056280F82B
:1013E0004C5000F0BFFF63681B6823B129462046BC
:1013F000BDE87040184770BD0278436880F86820E7
:1014000005221B6802700BB10421184770470000C9
:10141000436890F868201B6802700BB105211847DB
:101420007047000090F84C3070B5044613B10023AB
:1014300080F84C3004F15C02204601F0ADF863689E
:101440009B6863BB94F85C5015F0600615D194F866
:101450005D3005F07F0545EA032540F202339D42E9
:1014600000F00E815BD8022D00F0DC803FD8002D0B
:1014700000F08780012D00F0CF800021204601F090
:10148000F5FA0021204601F0E7FA63681B6813B102
:10149000062120469847062384F84C3070BD20462C
:1014A00098470028CED094F8632094F8623043EA3D
:1014B0000223626D934238BF636594F95C30656DB9
:1014C000002B4FF0200380F2FD80002D00F0EC8017
:1014D000092284F84C2083F311880021636D226D6A
:1014E0002046FFF757FF002383F3118870BDB5F541
:1014F000817F00F0B180B5F5407F49D0B5F5807FA0
:10150000BBD194F85E30012BB7D1B4F8643023F02E
:101510000203A4F8643026656665A665C3E740F259
:1015200001639D421ED8B5F5C06F3BD2B5F5A06FE3
:10153000A3D1B4F85C30B3F5A06F0ED194F85E304F
:10154000204684F8663000F065FF63681B6813B1BD
:1015500001212046984703232370002323656365F8
:10156000A365A0E7B5F5106F32D040F602439D4267
:1015700052D0B5F5006F80D104F1670323650123D4
:1015800024E004F16403A5652365022363658AE70B
:1015900094F85E30012B7FF470AFB4F8643043F000
:1015A0000203B6E794F861202046616894F8603041
:1015B0004D6843EA022394F85F1094F85E20A84730
:1015C00000283FF45AAF4368236503686365A4E7C6
:1015D0002378042B10D1202383F311882046FFF7B2
:1015E000B7FE86F311886368032184F867601B687F
:1015F00021700BB12046984794F85E30002BACD098
:1016000084F867300423237063681B68002BA4D020
:10161000022120469847A0E7374B236502236365E4
:1016200000239DE794F86010204611F0800F01F030
:101630000F010ED000F0A2FF012806D002287FF48F
:101640001CAF2E4B6065236567E72D4B65652365F1
:1016500063E700F085FFEFE794F85E30002B7FF43E
:101660000CAF94F8603013F00F013FF476AF1A0618
:10167000204602D501F00EFA6FE701F001FA6CE79F
:1016800094F85E30002B7FF4F8AE94F8603013F0DD
:101690000F013FF462AF1B06204602D501F0E6F9C8
:1016A0005BE701F0D9F958E7142284F84C2083F362
:1016B00011882B462A4629462046FFF759FE85F316
:1016C000118870BD5DB1152284F84C2083F3118818
:1016D0000021636D226D2046FFF74AFE03E70B22CF
:1016E00084F84C2083F311882B462A46294620464D
:1016F000FFF750FEE3E700BFB4350008AC35000843
:10170000B035000838B590F84C300446152B29D870
:10171000DFE803F03E28282828283E28280B29390E
:1017200028282828282828283E3E90F8631090F87A
:101730006220436D42EA01229A4214D9C268128A99
:10174000B3FBF2F502FB15356DB9202383F3118845
:101750002B462A462946FFF71DFE85F311880A23EA
:1017600084F84C3038BD142384F84C30202383F3A4
:101770001188002320461A461946FFF7F9FD002379
:1017800083F3118838BD836D03B198470023E7E7E1
:10179000002101F06BF90021204601F05DF963683A
:1017A0001B6813B10621204698470623D8E700009E
:1017B00090F84C20152A38B5044622D801239340CE
:1017C00040F6416213421DD113F480150FD19B02E4
:1017D00017D50B2380F84C30202383F311882B4638
:1017E0002A462946FFF7D6FD85F3118838BDC36820
:1017F0009B695B682BB9836D03B19847002384F81C
:101800004C3038BD002101F031F90021204601F0B3
:1018100023F963681B6813B1062120469847062305
:10182000EDE70000024B00221B605B609A6070478E
:1018300030260220002382680374054B1B689968D8
:101840009142FBD25A680360426010605860704752
:101850003026022008B5202383F31188037C032B54
:1018600005D0042B0DD02BB983F3118808BD436933
:1018700000221A604FF0FF334361FFF7DBFF0023C4
:10188000F2E790E80C001A6002685360F2E700008B
:10189000002382680374054B1B6899689142FBD84A
:1018A0005A6803604260106058607047302602201A
:1018B000054B196908741868026853601A6018614A
:1018C00001230374FEF730BD302602204B1C30B5D7
:1018D000054687B00A4C10D0236901A8094A00F0D8
:1018E000D3F82846FFF7E4FF049B13B101A800F0EA
:1018F00007F92369586907B030BDFFF7D9FFF8E74A
:10190000302602205518000838B50C4D04464161B8
:101910002B6981689A68914203D8BDE83840FFF787
:1019200089BF1846FFF786FF01232C610146237407
:101930002046BDE83840FEF7F7BC00BF3026022045
:10194000044B1A681B6990689B68984294BF0020FA
:10195000012070473026022010B5084C236820690A
:101960001A6854602260012223611A74FFF790FF05
:1019700001462069BDE81040FEF7D6BC30260220A3
:101980008260022202740022427470478368A3F1CD
:101990007C0243F80C2C026943F83C2C426943F862
:1019A000382C074A43F81C2CC268A3F1180043F8EE
:1019B000102C022203F8082C002203F8072C704791
:1019C0004103000810B5202383F31188FFF7DEFFE1
:1019D00000210446FFF798FF002383F31188204677
:1019E00010BD0000024B1B6958610F20FFF760BF5C
:1019F00030260220202383F31188FFF7F3BF000075
:101A000008B50146202383F311880820FFF75EFF05
:101A1000002383F3118808BD49B1064B42681B6956
:101A200018605A60136043600420FFF74FBF4FF007
:101A3000FF307047302602200368984206D01A68AB
:101A40000260506018465961FFF7F4BE704700000D
:101A500038B504460D462068844200D138BD03687D
:101A600023605C604561FFF7E5FEF4E7054B03F199
:101A700014025A619A614FF0FF32DA6100221A6251
:101A8000704700BF30260220F8B503614FF0804355
:101A9000C26002295C6A0646184B38BF02211A460A
:101AA0001F4652F8145F95420AD1586198611C6232
:101AB0000560456081600819BDE8F84001F0D8B9BB
:101AC000186AAB68241A0C1902D3E41A2D6804E0D2
:101AD0009C4202D2204401F0D9F9AB689C42F4D870
:101AE0006B68356073601E604FF0FF336E60B460EA
:101AF000A968091BA960FB61F8BD00BF3026022060
:101B000010B41B4C234653F8141F814210D0416877
:101B100002680A60026851609A424FF00001C16099
:101B200003D0936881680B4493605DF8044B704761
:101B30000A6800209A4262615360C86003D15DF870
:101B4000044B01F09DB9936888680344206A936050
:101B50004FF08042526A121A9342E6D9991A5DF800
:101B6000044B012998BF931C184401F08FB900BFA2
:101B70003026022000207047FEE70000704700007A
:101B80004FF0FF3070470000022906D0032906D02D
:101B90000129064818BF0020704705487047032AEE
:101BA0009ABF044800EBC20000207047843600084A
:101BB000383600083024022070B59AB00646084630
:101BC000144601AD294600F095F82846FFF736F98E
:101BD000C0B2431C5B0086E8180023700323023464
:101BE00004F8013C00231946DAB20234904201D8CD
:101BF0001AB070BDEA5C013304F8011C04F8022C31
:101C0000F2E7000008B5202383F311880348FFF7AB
:101C1000E1FA002383F3118808BD00BF702602207B
:101C200010B50446052916D8DFE801F0161503168D
:101C3000161D202383F311880E4A0121FFF76EFB46
:101C400020460D4A0221FFF769FB0C48FFF788FA8E
:101C5000002383F3118810BD202383F311880748E4
:101C6000FFF754FAF4E7202383F311880348FFF7C2
:101C70006BFAEDE7B8350008DC3500087026022065
:101C800038B50C4D0C4C2A460C4904F10800FFF7FE
:101C900093FF05F1CA0204F110000949FFF78CFF18
:101CA00005F5CA7204F118000649BDE83840FFF78F
:101CB00083BF00BF382B02203024022008360008E2
:101CC000123600081D36000870B5044608460D4659
:101CD000FFF7B4F8C6B22046013403780BB91846B2
:101CE00070BD32462946FFF793F80028F3D1012052
:101CF00070BD00002DE9F84F05460C46FFF79EF831
:101D00002B49C6B22846FFF7DFFF2A492846FFF7CE
:101D1000DBFF08B11036F6B2632E0DD8DFF89080E5
:101D2000DFF89090244FDFF898A0DFF898B02E7875
:101D300046B92670BDE8F88F29462046BDE8F84F21
:101D400001F0FABB252E2ED1072241462846FFF787
:101D50005FF870B9DBF800300735073444F8073C0A
:101D6000BBF8043024F8033C9BF8063004F8013C2F
:101D7000DDE7082249462846FFF74AF898B9A21C31
:101D80000E4B13F8011F023209095345C95D02F8D1
:101D9000041C197801F00F01C95D02F8031CF0D191
:101DA00018340835C3E7267001350134BFE700BF9A
:101DB000A43600081D360008B43600081FF4F01FD2
:101DC0002BF4F01FAC360008BFF34F8F024AD368E4
:101DD000DB03FCD4704700BF003C024008B5074B52
:101DE0001B7853B9FFF7F0FF054B1A69002A04DA94
:101DF000044A5A6002F188325A6008BD962D0220CA
:101E0000003C02402301674508B5054B1B7833B9F8
:101E1000FFF7DAFF034A136943F00043136108BD7B
:101E2000962D0220003C02400B2870B513D80B4AB7
:101E30000B4C137863B94FF000610A4E44F823103D
:101E400056F8235001330C2B2944F7D1012313708A
:101E500054F8200070BD002070BD00BFC82D0220C6
:101E6000982D0220C8360008014B53F82000704717
:101E7000C83600080C2070470B2810B5044601D95D
:101E8000002010BDFFF7D0FF064B53F82430184454
:101E9000C21A0BB9012010BD12680132F0D1043B07
:101EA000F6E700BFC83600080B2810B5044621D855
:101EB000FFF78AFFFFF792FF0F4AF323D360C300B7
:101EC000DBB243F4007343F002031361136943F47C
:101ED00080331361FFF778FFFFF7A6FF074B53F836
:101EE000241000F0DBF8FFF78FFF2046BDE810401C
:101EF000FFF7C2BF002010BD003C0240C8360008FA
:101F00002DE9F84312F0010315463FD18218B2F1D2
:101F1000026F3BD22B4B1B6813F0010336D0FFF747
:101F20005DFF294CF32340F20127E360FFF74CFFEC
:101F3000032D01D9830712D00F46401A224C40F2DC
:101F40000118EB1BC6190B44012B236924D823F07D
:101F500001032361FFF758FF0120BDE8F8832369DF
:101F600023F44073236123693B43236151F8046BDD
:101F70000660BFF34F8FFFF727FF03689E4208D02C
:101F8000236923F001032361FFF73EFF0020BDE832
:101F9000F883043D0430CBE723F44073B946236152
:101FA000236943EA0803236137F8023B3380BFF318
:101FB0004F8FFFF709FF3688B6B2B9F80030B34249
:101FC000BFD0DDE700380240003C0240084908B5B8
:101FD0000B7828B153B9FFF701FF01230B7008BD3F
:101FE00023B10870BDE80840FFF70EBF08BD00BF71
:101FF000962D022002440439064BD2B210B590420D
:1020000000D110BD441C00B253F8200041F8040F69
:10201000E0B2F4E750280040104B30B51C6F2404A8
:1020200007D41C6F44F400741C671C6F44F4004414
:102030001C670B4C024404392368D2B243F480730A
:102040002360084B904200D130BD441C51F8045F1E
:1020500000B243F82050E0B2F4E700BF003802407D
:10206000007000405028004007B5012201A900205F
:10207000FFF7C0FF019803B05DF804FB13B50446F9
:10208000FFF7F2FFA04206D002A90122002041F88A
:10209000044DFFF7C1FF02B010BD00000144BFF3C3
:1020A0004F8F064B884204D3BFF34F8FBFF36F8F20
:1020B0007047C3F85C022030F4E700BF00ED00E099
:1020C000034B1B689B0042BF0122024B1A707047F2
:1020D00074380240C92D0220014B1878704700BFA8
:1020E000C92D0220F0B5BFF34F8FBFF36F8F1D4B8B
:1020F0000021C3F85012BFF34F8FBFF36F8F5A699F
:1021000042F400325A61BFF34F8FBFF36F8FC3F8B1
:102110008410BFF34F8FD3F8802043F6E076C2F3EC
:10212000C904C2F34E32A507520102EA060E284640
:1021300021464EEA0007013900F14040C3F86072C1
:102140004F1CF6D1203A12F1200FEED1BFF34F8F82
:102150005A6942F480325A61BFF34F8FBFF36F8FD9
:10216000F0BD00BF00ED00E0FEE70000084A094BAB
:1021700009498B4204D3094A0021934205D3704791
:1021800052F8040F43F8040BF3E743F8041BF4E799
:10219000D43800085830022058300220583002202D
:1021A000036F002230B51146C46E9D684FF0FF30BA
:1021B00004EB421301329542C3F80019C3F8101919
:1021C000C3F80809C3F8001BC3F8101BC3F8080BB9
:1021D000EED24FF00113C4F81C3830BD890141F034
:1021E0002001016103699B06FCD4122000F0DABED5
:1021F000204B03EB80022DE9F047D2F80CE0461C9F
:10220000DD6EDEF8142005EB0636D2F800C005EBD3
:102210004018516861450BD30123D5F8342803FADF
:1022200000F022EA0000C5F834081846BDE8F0873F
:10223000ACEB0103BEF81040A34228BF2346D8F8F8
:102240001849A4B2B3EB840F10D894681F46A4F1C8
:10225000040959F804AF042FC6F800A001D9043FBF
:10226000F7E71C440B4494605360D2E70020BDE8BC
:10227000F08700BFCC2D022010B5054C2046FFF79B
:1022800029F84FF0A043E366024B236710BD00BF5F
:10229000CC2D02201C3700080378012B70B50546B1
:1022A00050D12A4BC46E98421BD1294B0E2143209A
:1022B0005A6B42F080025A635A6D42F080025A65AE
:1022C0005A6D5A6942F080025A615A6922F08002BE
:1022D0005A615B6900F0E8FB1E4BE3601E4BC4F8DB
:1022E00000380023EE6EC4F8003EC02323604FF494
:1022F0000413A3633369002BFCDA01230C20336140
:1023000000F050FE3369DB07FCD4122000F04AFED7
:102310003369002BFCDA00262846A660FFF740FF51
:102320006B68C4F81068DB68C4F81468C4F81C68EB
:102330004BB90A4BA3614FF0FF336361A36843F0CD
:102340000103A36070BD064BF4E700BFCC2D022053
:10235000003802404014004003002002003C30C01E
:10236000083C30C0F8B5C46E054600214FF0006649
:102370002046FFF733FF296F00234FF001128F68CB
:102380004FF0FF30C4F83438C4F81C2804EB431273
:1023900001339F42C2F80069C2F8006BC2F8080915
:1023A000C2F8080BF2D20B68EA6E6B676362102307
:1023B0001361166916F01006FBD1122000F0F2FD31
:1023C000D4F8003823F4FE63C4F80038A36943F45A
:1023D000402343F01003A3610923C4F81038C4F864
:1023E00014380A4BEB604FF0C043C4F8103B084B65
:1023F000C4F8003BC4F81069C4F800396B6F03F1EE
:10240000100243F480136A67A362F8BDF83600082F
:1024100040800010C26E90F86610D2F8003823F4A5
:10242000FE6343EA0113C2F8003870472DE9F0411A
:102430000EB20D4600EB8608D8F80C100F6807F0B6
:102440000303022B50D0032B50D03D4A3D4F012BAC
:1024500018BF1746C46E4FEA451E002205F1100C46
:1024600004EB0E03C3F8102B8A69002A40D04A8A75
:1024700005F158033A435B01E2500123D4F81C28CC
:1024800003FA0CF31343C4F81C38A64400234A692A
:10249000CEF8103905F13F03002A39D00A8A04EB3F
:1024A0008303898B9208012988BF4A43416F5618DC
:1024B00041EA02422946466720465A60FFF78EFEEF
:1024C000D8F80C301B8A43EA85531F4305F14803B3
:1024D0005B01E7500123D4F81C2803FA05F51543E6
:1024E000C4F81C58BDE8F081174FB3E7174FB1E7A8
:1024F00004EB4613D3F8002B22F40042C3F8002B60
:102500000123D4F81C2803FA0CF322EA0303BAE7E8
:1025100004EB83030E4A04EB461629465A60204614
:10252000FFF75CFED6F80039012223F4004302FADB
:1025300005F5C6F80039D4F81C3823EA0505CFE7BD
:1025400000800010008004100080081000800C1033
:1025500000040002026F12684267FFF721BE00000C
:102560005831C36E49015B5813F4004004D013F492
:10257000001F14BF01200220704700004831C36EC5
:1025800049015B5813F4004004D013F4001F14BF3A
:10259000012002207047000000EB8101CB68196A1E
:1025A0000B6813604B6853607047000000EB8103B9
:1025B00030B5DD68AA691368D36019B9402B84BFB0
:1025C000402313606B8A1468C26E1C4402EB4110F6
:1025D000013C09B2B4FBF3F46343033323F0030378
:1025E00043EAC44343F0C043C0F8103B2B6803F0F8
:1025F0000303012B0ED1D2F8083802EB411013F47B
:10260000807FD0F8003B14BF43F0805343F0005369
:10261000C0F8003B02EB4112D2F8003B43F0044308
:10262000C2F8003B30BD00002DE9F041244D0446C6
:10263000EE6E06EB4013D3F8087B3807C3F8087B2F
:102640000AD5D6F81438190706D505EB84032146B8
:102650002846DB685B689847FA072FD5D6F8143808
:10266000DB072BD505EB8403D968CCB98B69488A85
:102670005E68B6FBF0F200FB12628AB91868DA688D
:1026800090420DD2121A83E81400202383F311889C
:102690000B482146FFF78AFF84F31188BDE8F081DB
:1026A000012303FA04F26B8923EA02036B81CB68EE
:1026B00023B121460248BDE8F0411847BDE8F0814A
:1026C000CC2D022000EB81034A0170B5DD68C36E9A
:1026D0006C692668E66056BB1A444FF40020C2F8C5
:1026E00010092A6802F00302012A0AB20ED1D3F8B7
:1026F000080803EB421410F4807FD4F8000914BFDB
:1027000040F0805040F00050C4F8000903EB421242
:10271000D2F8000940F00440C2F800090122D3F8C1
:10272000340802FA01F10143C3F8341870BD19B935
:10273000402E84BF4020206020681A442E8A8419CD
:1027400040F00050013CB4FBF6F440EAC440C6E758
:10275000F8B504461E48C56E05EB4413D3F8086966
:10276000F107C3F8086917D5D5F81038DA0713D57B
:1027700000EB8403D9684B691F68DA68974218D266
:10278000D21B00271A605F60202383F31188214643
:10279000FFF798FF87F31188330617D50123D5F883
:1027A0003428A340134211D02046BDE8F840FFF77B
:1027B0001FBD012303FA04F2038923EA0203038104
:1027C0008B68002BE8D021469847E5E7F8BD00BFAD
:1027D000CC2D02209F482DE9F84FC56E04466E6946
:1027E000AB691E4016F4805F6E6105D0FEF7E4FD14
:1027F000BDE8F84F00F078BC002E12DAD5F8003EA4
:102800009B0705D0D5F8003E23F00303C5F8003E32
:10281000D5F804388F4823F00103C5F80438FEF7D3
:10282000F7FD370502D58B48FEF7E6FDB0040CD561
:10283000D5F8083813F0060FEB6823F470530CBF7B
:1028400043F4105343F4A053EB60310704D563689D
:10285000DB680BB17F489847F2026FD4B3020CD506
:10286000D4F86C8000274FF00109DFF8E8A1236F4E
:10287000F9B29B688B4280F09C80F70619D5E16E17
:102880000A6AC2F30A1702F00F0302F4F012B2F55B
:10289000802F00F0B580B2F5402F0AD104EB8303FE
:1028A00001F58051DB68186A00231A469F4240F008
:1028B0009C803303D5F818481DD5E70302D50020C6
:1028C000FFF7B2FEA50302D50120FFF7ADFE6003BE
:1028D00002D50220FFF7A8FE210302D50320FFF74F
:1028E000A3FEE20202D50420FFF79EFEA30202D55A
:1028F0000520FFF799FE77037FF57AAFE60702D54B
:102900000020FFF725FFA50702D50120FFF720FFD4
:10291000600702D50220FFF71BFF210702D5032025
:10292000FFF716FFE20602D50420FFF711FFA3060A
:102930007FF55EAF0520FFF70BFF59E7D4F86C80F9
:1029400000274FF00109DFF80CA1236F5FFA87FB26
:102950009B685B4582D308EB4B13D3F8002902F444
:102960004022B2F5802F22D1D3F80029002A1EDAA6
:10297000D3F8002942F09042C3F80029D3F8002987
:10298000002AFBDB5946E06EFFF728FC228909FA92
:102990000BF322EA0303238104EB8B03DB689B68C0
:1029A00013B15946504698475846FFF721FC013766
:1029B000CBE708EB4112D2F8003B03F44023B3F518
:1029C000802F10D1D2F8003B002B0CDA628909FA73
:1029D00001F322EA0303638104EB8103DB68DB6814
:1029E0000BB150469847013741E79C0700D10A6870
:1029F000072B03F101039EBF0270120A013055E755
:102A0000023301F5805104EB830252689069026839
:102A1000D0F808C04068A2EB000E00221046974292
:102A20000AD104EB830463689B699A683A449A600C
:102A30005A6817445F603CE712F0030F00D1086842
:102A4000964502F1010282BF8CF80000000A0CF1E9
:102A5000010CE4E7CC2D0220C36E03EB4111D1F849
:102A6000003B43F40013C1F8003B7047C36E03EB17
:102A70004111D1F8003943F40013C1F8003970470F
:102A8000C36E03EB4111D1F8003B23F40013C1F8EE
:102A9000003B7047C36E03EB4111D1F8003923F4BA
:102AA0000013C1F80039704700F1604300F01F02C5
:102AB0000901400903F56143C9B2800083F800139E
:102AC000012300F16040934000F56140C0F880317F
:102AD0000360704730B50433039C0172002104FB8E
:102AE0000325C361049B00600363059B4060C160D4
:102AF000426102618561046242628162C162436334
:102B000030BD00000022416AC260416101616FF086
:102B100001018262C262FEF79BBF00000369426945
:102B2000934203D1C2680AB100207047181D704754
:102B3000036919600021C2680132C260C26913448E
:102B400082699342036124BF436A0361FEF774BF45
:102B500038B504460D46E3683BB162690020131D99
:102B60001268A3621344E36238BD237A33B929465D
:102B70002046FEF751FF0028EDDA38BD6FF0010066
:102B8000FBE70000C368C269013BC36043691344AB
:102B900082699342436124BF436A43610023836295
:102BA000036B03B11847704770B52023044683F3C5
:102BB0001188866A3EB9FFF7CBFF054618B186F348
:102BC0001188284670BDA36AE26A13F8015B93423C
:102BD000A36202D32046FFF7D5FF002383F31188B9
:102BE000EFE700002DE9F84F04460E46904699465F
:102BF000202787F311880025AA46D4F828B0BBF116
:102C0000000F09D149462046FFF7A2FF20B18BF300
:102C100011882846BDE8F88FA16AA8EB050BE36A86
:102C20005B1A9B4528BF9B46BBF1400F1BD933461F
:102C300001F1400251F8040B914243F8040BF9D121
:102C4000A36A403640354033A362A26AE36A9A42DF
:102C500002D32046FFF796FF8AF311884545D8D264
:102C600087F31188C9E730465A46FEF7C7F8A36ACA
:102C70005E445D445B44A362E7E7000010B5029C3C
:102C800004330172C36103FB0421002300608362EB
:102C9000C362039B40600363049BC46042610261A2
:102CA000816104624262436310BD0000026A6FF0FA
:102CB0000101C260426A4261026100228262C26214
:102CC000FEF7C6BE436902699A4203D1C2680AB1DF
:102CD00000207047184650F8043B0B607047000016
:102CE000C3680021C2690133C36043691344826928
:102CF0009342436124BF436A4361FEF79DBE0000D7
:102D000038B504460D46E3683BB1236900201A1D1F
:102D1000A262E2691344E36238BD237A33B92946DB
:102D20002046FEF779FE0028EDDA38BD6FF001008D
:102D3000FBE7000003691960C268013AC260C2691A
:102D4000134482699342036124BF436A03610023F1
:102D50008362036B03B118477047000070B52023EE
:102D600004460E4683F31188856A35B91146FFF78C
:102D7000C7FF10B185F3118870BDA36A1E70A36AE6
:102D8000E26A01339342A36204D3E1692046043925
:102D9000FFF7D0FF002080F3118870BD2DE9F84FB8
:102DA00004460D4691469A464FF0200888F3118854
:102DB0000026B346A76A4FB951462046FFF7A0FF49
:102DC00020B187F311883046BDE8F88FA06AA9EBDF
:102DD0000603E76A3F1A9F4228BF1F46402F1BD9B0
:102DE00005F1400355F8042B9D4240F8042BF9D11E
:102DF000A36A40364033A362A26AE36A9A4204D3CC
:102E0000E16920460439FFF795FF8BF311884E45A1
:102E1000D9D288F31188CDE729463A46FDF7EEFF6F
:102E2000A36A3D443E443B44A362E5E7026943692B
:102E30009A4203D1C3681BB9184670470023FBE7C9
:102E4000836A002BF8D0043B9B1AF5D01360C3684B
:102E5000013BC360C3691A4483699A42026124BF7B
:102E6000436A0361002383620123E5E700F07EB932
:102E70004FF08043002258631A610222DA607047E3
:102E800000224FF08043DA60704700004FF080432B
:102E900058637047FEE7000010B5194CFEF7C2FCFE
:102EA000FEF7E4FD802217492046FEF769FD012365
:102EB00044F8180C0374144B144AD96821F4E061E7
:102EC0000904090C0A431249DA60CA6842F08072A8
:102ED000CA60104A1049C2F8B01F116841F00101E0
:102EE00011601022DA77202283F82220002383F356
:102EF000118862B60948BDE81040FEF763BD00BF07
:102F0000582602202837000800ED00E00003FA05EB
:102F1000F0ED00E0001000E055CEACC53037000801
:102F20002DE9F84F1E4C4FF00008656904F11407B5
:102F3000C1464FF08043266AAA685B6A9E1B964290
:102F40001CD34FF0200AAA68236AD5F80CB0B61A31
:102F5000134423622B68BB425F606361C5F80C8039
:102F600001D1FFF78DFF89F311882869D8478AF3CB
:102F700011886569AB689E42E5D2DAE76269BA42B8
:102F80000CD0916823628E1B9660A86802282CBF23
:102F90001818981CBDE8F84FFFF778BFBDE8F88F08
:102FA00030260220034B59685A68521A9042FBD8C7
:102FB000704700BF001000E04B6843608B6883607F
:102FC000CB68C3600B6943614B6903628B694362E1
:102FD0000B6803607047000008B5274B40F2FF7193
:102FE00026481A690A431A611A6922F4FF6222F01C
:102FF00007021A611A691A6B0A431A631A6D0A43A7
:103000001A651F4A1B6D1146FFF7D6FF1D4802F1D6
:103010001C01FFF7D1FF1C4802F13801FFF7CCFF7C
:103020001A4802F15401FFF7C7FF194802F1700175
:10303000FFF7C2FF174802F18C01FFF7BDFF1648EA
:1030400002F1A801FFF7B8FF144802F1C401FFF72D
:10305000B3FF134802F1E001FFF7AEFF114802F1A0
:10306000FC01FFF7A9FF104802F58C71FFF7A4FFE0
:10307000BDE8084000F0DCB8003802400000024023
:10308000503700080004024000080240000C0240D3
:10309000001002400014024000180240001C0240D0
:1030A00000200240002402400028024008B500F041
:1030B00033FAFFF7F1FEFFF703F8BDE80840FEF72B
:1030C000DFBD000070470000064A536823F001038B
:1030D0005360EFF30983683383F30988002383F394
:1030E0001188704730EF00E010B5202383F311887A
:1030F000104B5B6813F4006318D0F1EE103AEFF355
:1031000009844FF0807344F84C3C0B4BDB6844F867
:10311000083CA4F1680383F30988FEF711FC18B199
:10312000064B44F8503C10BD054BFAE783F3118879
:1031300010BD00BF00ED00E030EF00E051030008DB
:10314000540300084FF080431A69920710B508D560
:1031500000241C61202383F31188FFF7E1FE84F330
:103160001188BDE81040FFF7BFBF0000104B0821D9
:103170001C201A6C42F001021A641A6E42F001021D
:103180001A660C4A1B6E936843F0010393604FF07C
:1031900080436B229A624FF0FF32DA6200229A611A
:1031A0005A63DA605A6001225A611A60FFF77CBCE8
:1031B00000380240002004E01B4B4FF0FF3000219C
:1031C0001A696FEA42526FEA52521A611A69C2F3DF
:1031D0000A021A611A695A6958615A6959615A6929
:1031E0001A6A62F080521A621A6A02F080521A62F7
:1031F0001A6A5A6A58625A6A59625A6A0B4A1068BD
:1032000040F480701060186F00F44070B0F5007FDB
:1032100003D04FF4803018671967536823F40073A4
:10322000536000F059B900BF003802400070004000
:10323000354B4FF44041354A1A64354A11601A68DB
:1032400042F001021A601A689207FCD59A6822F0CF
:1032500003029A602C4B19469A6812F00C02FBD1BB
:10326000186800F0F90018609A601A6842F4803219
:103270001A600B689B03FCD54B6F43F001034B674F
:10328000214B5A6F9007FCD5224A5A601A6842F0C7
:1032900080721A601E4B1A4659684904FCD5196899
:1032A00041F4803119605368D803FCD5136843F4A6
:1032B00000331360164A53689903FCD5124B1A6801
:1032C0009201FCD5144A40F207319A6040F2011293
:1032D000C3F88C200022C3F89020104A11609A682D
:1032E00042F002029A60084B9A6802F00C02082A27
:1032F000FAD15A6C42F480425A645A6E42F48042C7
:103300005A665B6E704700BF003802400004001030
:1033100000700040086C400900948838003C02406E
:10332000084A08B5536911680B4003F00103536163
:1033300023B1054A13680BB150689847BDE80840AF
:10334000FFF7D2BE003C0140B0250220084A08B574
:10335000536911680B4003F00203536123B1054A1E
:1033600093680BB1D0689847BDE80840FFF7BCBE32
:10337000003C0140B0250220084A08B55369116895
:103380000B4003F00403536123B1054A13690BB1E9
:1033900050699847BDE80840FFF7A6BE003C0140D1
:1033A000B0250220084A08B5536911680B4003F0A4
:1033B0000803536123B1054A93690BB1D06998475B
:1033C000BDE80840FFF790BE003C0140B025022058
:1033D000084A08B5536911680B4003F010035361A4
:1033E00023B1054A136A0BB1506A9847BDE80840FB
:1033F000FFF77ABE003C0140B0250220174B10B504
:103400005C691A68144004F478725A61A30604D502
:10341000134A936A0BB1D06A9847600604D5104AE4
:10342000136B0BB1506B9847210604D50C4A936B74
:103430000BB1D06B9847E20504D5094A136C0BB168
:10344000506C9847A30504D5054A936C0BB1D06C1A
:103450009847BDE81040FFF747BE00BF003C014061
:10346000B02502201A4B10B55C691A68144004F4A8
:103470007C425A61620504D5164A136D0BB1506D3A
:103480009847230504D5134A936D0BB1D06D984727
:10349000E00404D50F4A136E0BB1506E9847A10497
:1034A00004D50C4A936E0BB1D06E9847620404D5D4
:1034B000084A136F0BB1506F9847230404D5054A8F
:1034C000936F0BB1D06F9847BDE81040FFF70CBE6B
:1034D000003C0140B0250220062108B50846FFF750
:1034E000E3FA06210720FFF7DFFA06210820FFF79D
:1034F000DBFA06210920FFF7D7FA06210A20FFF799
:10350000D3FA06211720FFF7CFFA06212820BDE8BD
:103510000840FFF7C9BA000008B5FFF74DFEFDF7F8
:1035200027FDFDF7D5FEFDF7A9FDFFF7CBFDBDE8B3
:103530000840FFF79BBC0000034611F8012B03F87D
:10354000012B002AF9D1704712101213121100003A
:103550000010410001105A0053544D3332463F3F92
:103560003F3F3F3F0053544D333246375B347C3549
:103570005D780053544D333246375B367C375D7887
:103580000000000000000000F50F0008E10F000837
:103590001D1000080910000815100008011000088F
:1035A000ED0F0008D90F0008791000080000000096
:1035B0000100000000000000020000000000000008
:1035C000211200088912000840004000082B022048
:1035D000182B022002000000000000000300000081
:1035E00000000000CD1200080000000010000000E4
:1035F000282B022000000000010000000000000055
:10360000CC2D0220010102004172647550696C6F7B
:10361000740025424F415244252D424C002553450C
:103620005249414C25000000211C0008891B00085C
:103630008D110008051C00084300000040360008FA
:1036400009024300020100C0320904000001020225
:1036500001000524001001052401000104240202D8
:103660000524060001070582030800FF0904010084
:10367000020A000000070501024000000705810260
:1036800040000000120000008C36000812011001FA
:10369000020000400912415700020102030100002C
:1036A0000403090425424F41524425005239506910
:1036B0006C6F74003031323334353637383941422B
:1036C00043444546000000000080000000800000E8
:1036D00000800000008000000000020000000400E4
:1036E00000000400000004000000040000000400CA
:1036F0000000040000000400000000002514000881
:1037000005170008B117000840004000442E0220B1
:10371000442E022001000000542E022080000000F0
:1037200040010000050000006D61696E00000000AE
:1037300048370008602E02205830022001000000A7
:10374000952E00080000000069646C650000000010
:103750000401806A00000000AAAAAAAA040100408D
:10376000FFFF00000000000000A00A0000000001B0
:1037700000000000AAAAAAAA00000001FFFF0000A2
:103780000000000000000000000000000000000039
:10379000AAAAAAAA00000000FFFF00000000000083
:1037A000000000000000000000000000AAAAAAAA71
:1037B00000000000FFFF000000000000000000000B
:1037C0000101000000000000AAAAAAAA000100004E
:1037D000FEFF0000000000000000000000000000EC
:1037E00000000000AAAAAAAA00000000FFFF000033
:1037F00000000000000000000000000000000000C9
:10380000AAAAAAAA00000000FFFF00000000000012
:10381000000000000000000000000000AAAAAAAA00
:1038200000000000FFFF000000000000000000009A
:103830000000000000000000AAAAAAAA00000000E0
:10384000FFFF00000000000000000000000000007A
:103850000000000000000000000000000000000068
:103860000000000000000000000000000000000058
:103870000000000000000000000000000000000048
:103880000000000000000000FF0000000000000039
:10389000583500083F000000490400006535000865
:1038A0003F00000051040000733500083F00000095
:1038B000009600000000080004000000A036000888
:1038C00000000000000000000000000000000000F8
:0838D0000000000000000000F0
:00000001FF
